 touch

 Timestamp is 4da293ae (Mon Apr 11 17:37:50 2011)

 Preferred load address is 10000000

 Start         Length     Name                   Class
 0001:00000000 00000112H .rdata                  CODE
 0001:00000114 00000022H .rdata$debug            CODE
 0001:00000138 00002490H .text                   CODE
 0001:000025c8 00000014H .xdata                  CODE
 0001:000025dc 00000014H .idata$2                CODE
 0001:000025f0 00000014H .idata$3                CODE
 0001:00002604 00000074H .idata$4                CODE
 0001:00002678 0000000cH .idata$6                CODE
 0001:00002690 00000161H .edata                  CODE
 0002:00000000 00000074H .idata$5                DATA
 0002:00000078 000000d4H .data                   DATA
 0002:00000160 0000016cH .bss                    DATA
 0003:00000000 00000150H .pdata                  DATA

  Address         Publics by Value              Rva+Base       Lib:Object

 0000:00000000       ___safe_se_handler_table   00000000     <absolute>
 0000:00000000       ___safe_se_handler_count   00000000     <absolute>
 0001:0000001c       MIN_CAL_COUNT              1000101c     touch.obj
 0001:00000020       ??_C@_1M@EPBPGMBG@?$AAA?$AAD?$AAC?$AA1?$AA?3?$AA?$AA@ 10001020     touch.obj
 0001:0000002c       ??_C@_1BI@KKLLCJMC@?$AAM?$AAa?$AAx?$AAC?$AAa?$AAl?$AAE?$AAr?$AAr?$AAo?$AAr?$AA?$AA@ 1000102c     tch_cal:calibrat.obj
 0001:00000044       ??_C@_1DC@PPKDPGKC@?$AAH?$AAA?$AAR?$AAD?$AAW?$AAA?$AAR?$AAE?$AA?2?$AAD?$AAE?$AAV?$AAI?$AAC?$AAE?$AAM?$AAA?$AAP?$AA?2?$AAT?$AAO?$AAU?$AAC?$AAH?$AA?$AA@ 10001044     tch_cal:calibrat.obj
 0001:00000078       ??_C@_1CA@IHOLOKEO@?$AAH?$AAi?$AAg?$AAh?$AAP?$AAr?$AAi?$AAo?$AAr?$AAi?$AAt?$AAy?$AA2?$AA5?$AA6?$AA?$AA@ 10001078     tchmdd:tchmain.obj
 0001:00000098       ??_C@_1BI@BHLBGEOK@?$AAP?$AAr?$AAi?$AAo?$AAr?$AAi?$AAt?$AAy?$AA2?$AA5?$AA6?$AA?$AA@ 10001098     tchmdd:tchmain.obj
 0001:000000b0       ??_C@_1CO@HCHNLANK@?$AA?2?$AAD?$AAr?$AAi?$AAv?$AAe?$AAr?$AAs?$AA?2?$AAB?$AAu?$AAi?$AAl?$AAt?$AAI?$AAn?$AA?2?$AAT?$AAo?$AAu?$AAc?$AAh?$AA?$AA@ 100010b0     tchmdd:tchmain.obj
 0001:000000e0       ??_C@_1BM@IOLIHJIC@?$AAA?$AAc?$AAt?$AAi?$AAv?$AAi?$AAt?$AAy?$AAE?$AAv?$AAe?$AAn?$AAt?$AA?$AA@ 100010e0     tchmdd:tchmain.obj
 0001:000000fc       ??_C@_1BG@JBGCDLHB@?$AAS?$AAy?$AAs?$AAt?$AAe?$AAm?$AA?2?$AAG?$AAW?$AAE?$AA?$AA@ 100010fc     tchmdd:tchmain.obj
 0001:00000138       ?TouchDriverCalibrationPointGet@@YAHPAUTPDC_CALIBRATION_POINT@@@Z 10001138 f   touch.obj
 0001:00000208       DdsiTouchPanelDetach       10001208 f   touch.obj
 0001:00000278       DdsiTouchPanelDisable      10001278 f   touch.obj
 0001:0000028c       DdsiTouchPanelEnable       1000128c f   touch.obj
 0001:000002ac       DdsiTouchPanelGetDeviceCaps 100012ac f   touch.obj
 0001:00000338       ?FilterSamples@@YAHPAUT_POSITION@@KK0@Z 10001338 f   touch.obj
 0001:00000470       DdsiTouchPanelGetPoint     10001470 f   touch.obj
 0001:00000674       DdsiTouchPanelPowerHandler 10001674 f   touch.obj
 0001:000006a8       DdsiTouchPanelSetMode      100016a8 f   touch.obj
 0001:000006dc       DdsiTouchPanelAttach       100016dc f   touch.obj
 0001:00000868       ComputeMatrix33            10001868 f   tch_cal:calibrat.obj
 0001:000009a8       TouchPanelCalibrateAPoint  100019a8 f   tch_cal:calibrat.obj
 0001:00000a54       ErrorAnalysis              10001a54 f   tch_cal:calibrat.obj
 0001:00000b80       TouchPanelSetCalibration   10001b80 f   tch_cal:calibrat.obj
 0001:00001140       LargeNumSet                10002140 f   tch_cal:largenum.obj
 0001:00001180       IsLargeNumNotZero          10002180 f   tch_cal:largenum.obj
 0001:000011b0       IsLargeNumNegative         100021b0 f   tch_cal:largenum.obj
 0001:000011c4       IsLargeNumMagGreaterThan   100021c4 f   tch_cal:largenum.obj
 0001:00001208       LargeNumMagInc             10002208 f   tch_cal:largenum.obj
 0001:00001238       LargeNumMagAdd             10002238 f   tch_cal:largenum.obj
 0001:000012a0       LargeNumMagSub             100022a0 f   tch_cal:largenum.obj
 0001:0000130c       LargeNumAdd                1000230c f   tch_cal:largenum.obj
 0001:000013b8       LargeNumSub                100023b8 f   tch_cal:largenum.obj
 0001:00001464       LargeNumMulUint32          10002464 f   tch_cal:largenum.obj
 0001:000014c8       LargeNumMult               100024c8 f   tch_cal:largenum.obj
 0001:00001620       LargeNumSignedFormat       10002620 f   tch_cal:largenum.obj
 0001:00001664       LargeNumRAShift            10002664 f   tch_cal:largenum.obj
 0001:00001748       LargeNumDivInt32           10002748 f   tch_cal:largenum.obj
 0001:00001864       LargeNumBits               10002864 f   tch_cal:largenum.obj
 0001:000018c4       TouchPanelDllEntry         100028c4 f   tchmdd:tchbasic.obj
 0001:00001d24       TouchPanelGetDeviceCaps    10002d24 f   tchmdd:tchmain.obj
 0001:00001d8c       TouchPanelSetMode          10002d8c f   tchmdd:tchmain.obj
 0001:00001e14       TouchPanelPowerHandler     10002e14 f   tchmdd:tchmain.obj
 0001:00001e18       TouchPanelEnable           10002e18 f   tchmdd:tchmain.obj
 0001:00002040       TouchPanelDisable          10003040 f   tchmdd:tchmain.obj
 0001:0000215c       TouchPanelReadCalibrationPoint 1000315c f   tchmdd:tchmain.obj
 0001:00002320       TouchPanelReadCalibrationAbort 10003320 f   tchmdd:tchmain.obj
 0001:0000236c       SetLastError               1000336c f   coredll:COREDLL.dll
 0001:0000237c       KernelIoControl            1000337c f   coredll:COREDLL.dll
 0001:0000238c       CloseHandle                1000338c f   coredll:COREDLL.dll
 0001:0000239c       InterruptMask              1000339c f   coredll:COREDLL.dll
 0001:000023ac       InterruptDone              100033ac f   coredll:COREDLL.dll
 0001:000023bc       DeviceIoControl            100033bc f   coredll:COREDLL.dll
 0001:000023cc       CreateFileW                100033cc f   coredll:COREDLL.dll
 0001:000023dc       RegCloseKey                100033dc f   coredll:COREDLL.dll
 0001:000023ec       RegQueryValueExW           100033ec f   coredll:COREDLL.dll
 0001:000023fc       RegOpenKeyExW              100033fc f   coredll:COREDLL.dll
 0001:0000240c       DisableThreadLibraryCalls  1000340c f   coredll:COREDLL.dll
 0001:0000241c       EventModify                1000341c f   coredll:COREDLL.dll
 0001:0000242c       InitializeCriticalSection  1000342c f   coredll:COREDLL.dll
 0001:0000243c       CreateEventW               1000343c f   coredll:COREDLL.dll
 0001:0000244c       ExitThread                 1000344c f   coredll:COREDLL.dll
 0001:0000245c       GetTickCount               1000345c f   coredll:COREDLL.dll
 0001:0000246c       LeaveCriticalSection       1000346c f   coredll:COREDLL.dll
 0001:0000247c       EnterCriticalSection       1000347c f   coredll:COREDLL.dll
 0001:0000248c       WaitForSingleObject        1000348c f   coredll:COREDLL.dll
 0001:0000249c       CeSetThreadPriority        1000349c f   coredll:COREDLL.dll
 0001:000024ac       CreateThread               100034ac f   coredll:COREDLL.dll
 0001:000024bc       InterruptInitialize        100034bc f   coredll:COREDLL.dll
 0001:000024cc       InterruptDisable           100034cc f   coredll:COREDLL.dll
 0001:000024dc       DeleteCriticalSection      100034dc f   coredll:COREDLL.dll
 0001:000024ec       OpenEventW                 100034ec f   coredll:COREDLL.dll
 0001:000024fc       __GSHandlerCheckCommon     100034fc f   corelib0:gshandler.obj
 0001:00002534       __GSHandlerCheck           10003534 f   corelib0:gshandler.obj
 0001:00002554       __security_check_cookie    10003554 f   corelib0:armsecgs.obj
 0001:00002564       __gsfailure                10003564     corelib0:armsecgs.obj
 0001:000025a8       __rt_udiv                  100035a8 f   corelib1:COREDLL.dll
 0001:000025b8       __report_gsfailure         100035b8 f   corelib1:COREDLL.dll
 0001:000025dc       __IMPORT_DESCRIPTOR_COREDLL 100035dc     coredll:COREDLL.dll
 0001:000025f0       __NULL_IMPORT_DESCRIPTOR   100035f0     coredll:COREDLL.dll
 0002:00000000       __imp_SetLastError         10004000     coredll:COREDLL.dll
 0002:00000004       __imp_KernelIoControl      10004004     coredll:COREDLL.dll
 0002:00000008       __imp_CloseHandle          10004008     coredll:COREDLL.dll
 0002:0000000c       __imp_InterruptMask        1000400c     coredll:COREDLL.dll
 0002:00000010       __imp_InterruptDone        10004010     coredll:COREDLL.dll
 0002:00000014       __imp_DeviceIoControl      10004014     coredll:COREDLL.dll
 0002:00000018       __imp_CreateFileW          10004018     coredll:COREDLL.dll
 0002:0000001c       __imp_RegCloseKey          1000401c     coredll:COREDLL.dll
 0002:00000020       __imp_RegQueryValueExW     10004020     coredll:COREDLL.dll
 0002:00000024       __imp_RegOpenKeyExW        10004024     coredll:COREDLL.dll
 0002:00000028       __imp_DisableThreadLibraryCalls 10004028     coredll:COREDLL.dll
 0002:0000002c       __imp_EventModify          1000402c     coredll:COREDLL.dll
 0002:00000030       __imp_InitializeCriticalSection 10004030     coredll:COREDLL.dll
 0002:00000034       __imp_CreateEventW         10004034     coredll:COREDLL.dll
 0002:00000038       __imp_ExitThread           10004038     coredll:COREDLL.dll
 0002:0000003c       __imp_GetTickCount         1000403c     coredll:COREDLL.dll
 0002:00000040       __imp_LeaveCriticalSection 10004040     coredll:COREDLL.dll
 0002:00000044       __imp_EnterCriticalSection 10004044     coredll:COREDLL.dll
 0002:00000048       __imp_WaitForSingleObject  10004048     coredll:COREDLL.dll
 0002:0000004c       __imp_CeSetThreadPriority  1000404c     coredll:COREDLL.dll
 0002:00000050       __imp_CreateThread         10004050     coredll:COREDLL.dll
 0002:00000054       __imp_InterruptInitialize  10004054     coredll:COREDLL.dll
 0002:00000058       __imp_InterruptDisable     10004058     coredll:COREDLL.dll
 0002:0000005c       __imp_DeleteCriticalSection 1000405c     coredll:COREDLL.dll
 0002:00000060       __imp_OpenEventW           10004060     coredll:COREDLL.dll
 0002:00000064       __imp___rt_udiv            10004064     corelib1:COREDLL.dll
 0002:00000068       __imp___rt_sdiv            10004068     corelib1:COREDLL.dll
 0002:0000006c       __imp___report_gsfailure   1000406c     corelib1:COREDLL.dll
 0002:00000070       \177COREDLL_NULL_THUNK_DATA 10004070     coredll:COREDLL.dll
 0002:00000078       gIntrTouch                 10004078     touch.obj
 0002:00000140       gdwTouchIstTimeout         10004140     tchmdd:tchmain.obj
 0002:00000144       __security_cookie          10004144     corelib0:seccinit.obj
 0002:00000148       __security_cookie_complement 10004148     corelib0:seccinit.obj
 0002:00000164       gIntrTouchChanged          10004164     touch.obj
 0002:00000248       v_pfnCgrCallback           10004248     tchmdd:tchbasic.obj
 0002:00000274       _bTchThreadHighPriority    10004274     tchmdd:tchmain.obj
 0002:00000278       hThread                    10004278     tchmdd:tchmain.obj
 0002:00000280       v_pfnPointCallback         10004280     <common>
 0002:00000284       CalibrationState           10004284     <common>
 0002:00000288       ghevCalibrationActivity    10004288     <common>
 0002:0000028c       culReferenceCount          1000428c     <common>
 0002:00000290       DisplayHeight              10004290     <common>
 0002:000002a0       csMutex                    100042a0     <common>
 0002:000002b4       hTouchPanelEvent           100042b4     <common>
 0002:000002b8       hCalibrationSampleAvailable 100042b8     <common>
 0002:000002bc       DisplayWidth               100042bc     <common>
 0002:000002c0       lCalibrationYCoord         100042c0     <common>
 0002:000002c4       lCalibrationXCoord         100042c4     <common>
 0002:000002c8       v_pfnCgrPointCallback      100042c8     <common>

 entry point at        0001:000018c4

 Static symbols

 0001:00001908       TouchPanelpISR             10002908 f   tchmdd:tchmain.obj
 0001:00001c60       TouchPanelpGetPriority     10002c60 f   tchmdd:tchmain.obj
